:020000040000FA
:0600000000008A018C28BB
:08000800FD000308FE00DB30DF
:1000100081070B11F10A0319F10A71087507F60D32
:1000200071087407F60D71087307F60D71087207F1
:10003000760D701B030177068700701D282870114C
:100040002708F2002808F3002908F4002A08F50020
:10005000F80B38281A30F800F90B38280508023A4E
:10006000F01802388500FA0B3828F014F01E7017CB
:100070007E088300FD0E7D0E0900A60194088C1EEB
:100080003F28171D3E2814088C1E442817194328A2
:100090001408031D3E280630FA00260FA6008C1E09
:1000A0004F2817193D281408A700260B4D28F010DB
:1000B00070138C1E592817193D281408A8008C1E8F
:1000C0005F2817193D281408A9008C1E65281719E8
:1000D0003D281408AA00701E74288C1E6D2817195C
:1000E0003D281408AB001A29F01D8628FF30A71FF1
:1000F0000030A700FF30A81F0030A800FF30A91F64
:100100000030A900FF30AA1F0030AA007015CC20D3
:10011000013E031D48293D2807309900831603132B
:10012000910170308F000F1D932800308100FD3049
:100130008500313095008312031301309300920142
:1001400091152030840080018008031D4629840A0F
:10015000841FA3280630FA00C4207708870083167E
:100160000313E030870083120313701AB828CD20E0
:10017000DB3081008B160B118B1797019717171621
:100180001408960185143D28F701051EF709851A04
:1001900008007016FC0AA401FF3483160313103004
:1001A0009B001C141A08A4009B0A1C149A1BF0152F
:1001B0009B0A1C149A1BF016831203130800831663
:1001C00003139B019C131C141A08FB009B0A1C14AC
:1001D0001A08FC008312031308008316031300306F
:1001E0009B007B08F9209B0A7C08F92083120313EB
:1001F000080083160313FE01FD009A009C131C15D2
:1002000055309D00AA309D009C1400009C180529C3
:1002100008001C141A087D0603190800FE0A7E084F
:10022000FB3E031944297D08FD288030FF3E031D55
:10023000162908008B018B0185102708FB00280870
:10024000FC00ED208316031310309B008312031370
:100250000030A91BFF30F920831603139B0A831279
:1002600003130030AA1BFF30F920831603139B0AE7
:10027000831203130030AB1BFF30F92002304B29EF
:1002800003304B2904304B2905304B2906304B29CC
:100290008B1308304B2983120313A3002308A200F9
:1002A0008514582185105A21A20B50295C214E2912
:1002B00003305D2909305D291430A100A0019F3071
:1002C000013E031C6029A00B5F29A10B5F290800D8
:02400E00E43399
:0442000000000100B9
:0642200000000000000098
:104230002034343420344334683461346E346E3482
:1042400065346C34203444344D345834353431348E
:1042500032342034503457344D34203444347234A2
:104260006934763465347234203420345634313431
:104270002E3431342E3432342034573465346234A1
:104280002034443465346D346F3420342034703439
:1042900069346334703472346F346A34653463342F
:1042A000743473342E346F34723467342E3475346E
:1042B0006B342034203428346334293420343234AD
:1042C0003034303439342034503465347434653407
:1042D0002034473472346934663466346934743453
:0642E00068347334203441
:00000001FF
